:020000040000FA
:020000001328C3
:08000800DE00030EDF0083128D
:100010000408AB00F3212B0884005F0E8300DE0E82
:100020005E0E0B11090083128501870107309900CC
:1000300083169101831609308500003087008316EE
:100040006400C0308100831620308B008312A90128
:100050008B17C0280F3982073034313432343334AF
:100060003434353436343734383439344134423426
:10007000433444344534463408000F398207BB34D6
:100080002834E334EA347834DA34DB342A34FB3489
:10009000FA347B34D9349334E934D33453340800FC
:1000A0000F398207653467346D346F3475347734B3
:1000B0007D347F34E534E734ED34EF34F534F73410
:1000C000FD34FF34080003398207BF34DF34FB34CA
:1000D000FE3408000739820780344034203410345D
:1000E0000834043402340134080003398207003430
:1000F0000034003401340800033982073234643498
:10010000FA34F434080007398207FF34FF34FF342F
:10011000FF34003408341034183408006722AF006C
:100120002F08031908002F038320AF00AF1F9B285F
:10013000AC01AD01080053082F041F398207F028D5
:10014000F42802290E29BF28BF28BF28BF28192953
:10015000222927292C29BF28BF28BF28BF287E296C
:100160007429BF286A29BF28BF28BF28BF2878293B
:100170007029BF286329BF28BF28BF28BF280800CF
:10018000EE22AC01AD01AE01D301D401D9010D3095
:10019000CA00BB30CB00A030CC000130C7003830E3
:1001A000C8008030C9000130C4008630C500A030CE
:1001B000C600CD01CE013230CF00D6015510D5108A
:1001C0005515871207128711D20152145216432176
:1001D0009B30B0009A21D2185B2361238E20EE2839
:1001E000D30AF230B0000800D30ADA30B000D130C0
:1001F000B100D330B2007330B300B401B501521175
:10020000A7210800D30A8030D4000430B400B10123
:100210009A21A3217C236B228A230800D3019B30DF
:10022000B0000430B400D4017C236B228A239A21CD
:100230000800521A9329D21A8E29521B8929D21BDF
:1002400084290800521919295215A3214329D60AD5
:100250005619D601A72108005908D700FC30D70D40
:10026000D70DD705D401C0014408C1004508C2001C
:100270004608C300403084000430D823E521E5213E
:100280008030D40008005908D700FC30D70DD70DB6
:10029000D705403084000430E023C01B5B294108AF
:1002A000C4004208C5004308C6007C236B228A2391
:1002B0009A21612308004030B200B300B400B500B9
:1002C000B600B70008001030D90A59060319D90141
:1002D000A32108000F30D903D91BD900A32108009E
:1002E000521D080063214329521D08006A21432939
:1002F0005214C222D2185B23612308005210C2227A
:10030000D2185B2361230800D2135213D212521663
:100310009729D2175213D21252129729D213521779
:10032000D21252129729D2135213D2165212871296
:10033000071287110030D21AC830521BC130D21BAD
:10034000C930B100080059083D20B0000800CD01B7
:1003500056087520CE0056087C20CF0083236B22E0
:1003600042083D20B500430E3D20B60043083D2025
:10037000B7000800A500250E2A20CC212E30CC2164
:1003800025082A20CC210800A500250E2A20CC21F2
:1003900025082A20CC2108008B13A1000830A000DA
:1003A0008514DF21A10C03188510031C8514A00BF4
:1003B000D129DF2185108B17DF21DF2100341E308A
:1003C000A2000000A20BE2290034FE30A300EA30B4
:1003D000A40000000000000000000000A30BE929B9
:1003E000A40BE9290034D21EFA298719F9298715A7
:1003F000FA2987110000521F022A071A012A07163C
:10040000022A07120000D21F0A2A871A092A871611
:100410000A2A87120000DA0ADA1D0800DA01AA0A9D
:10042000AA1E192A29086A2054050319192A03014A
:100430001D2A3030290784000008A8005020A6009B
:10044000A80CA80CA80CA80C28085020A700290864
:1004500063202919A705291DA6050830A800A60DA7
:1004600003180515031C051107100714A80B2F2AE4
:100470000830A800A70D03180515031C0511071067
:100480000714A80B3A2A2908A800A80AA90AA9193A
:10049000A90185195F2A2C08031D532A2808AC00DE
:1004A000AD00AE01662A28082C06031D662AAE0A96
:1004B000AE1D662A0730AE002808AD00662A2C085B
:1004C0000319662A28082C060319AC0108002D0818
:1004D000031DAD01080003101830B900C001C101AF
:1004E000C201C301BF0DBE0DBD0DC30DC20DC10DB7
:1004F000C00DB90B7C2A003443308400892242307D
:10050000840089224130840089224030840089227D
:10051000722A03300007B800B81980003030000795
:10052000B800B81B800000341830B900B801BF0D06
:10053000BE0DBD0DB80D0318A12A3C083802031CDE
:10054000A42A3C08B8020314C20DC10DC00DB90B9A
:10055000972A0034B9223C08BF07031CB22ABE0AFE
:100560000319BD0A3B08BE070318BD0A3A08BD07B8
:100570000034BC09BB09BA09BC0F0034BB0F0034FE
:10058000BA0A0034D214521CD02A4A08BD004B08C3
:10059000BE004C08BF007523AA22BD1B0134DA2A15
:1005A0007C234708BA004808BB004908BC00AA22BF
:1005B000BD1B01347C234D08BA004E08BB004F0818
:1005C000BC005218E52AAA22E62AAB223D08C40044
:1005D0003E08C5003F08C600D21000340715871436
:1005E000080007158714000000000000000000004C
:1005F0000000871000000000000000000000000064
:100600000711080087100715000000000000000017
:100610000000000087140800D1000830D000D10D80
:1006200003188714031C87101723D00B0F2B00000F
:10063000000000000000000000000715000000009E
:100640000000000000000000071108007C23323089
:10065000BC009422F122C6300C2341080C2342082E
:100660000C2388300C230230D51804305519013082
:100670000C23022308000330BD000D30BE000E30F5
:10068000BF007523AA22BD1B492B5514D510551147
:1006900008000730BD00A030BE00EE30BF0075235B
:1006A000AA22BD1B572B5510D51455110800551003
:1006B000D51055150800521C5F2B5210080052141B
:1006C00008003B2326237C236B228A230D30CC2178
:1006D0000A30CC214630CC212030CC214108C42125
:1006E0004208BA214308C42108004408BA0045085A
:1006F000BB004608BC0008004408BD004508BE0019
:100700004608BF0008004D08BD004E08BE004F0857
:10071000BF000800410E3D20B20041083D20B3005B
:10072000420E3D200438B40042083D20B500430E7F
:100730003D20B60043083D20B700BB303206031908
:10074000B2010800831203135708831603139B009A
:10075000831603131C14831603131A08831203133E
:10076000D800831603131C14831603131A0883126C
:100770000313D806031DA22B0800831603139C182D
:10078000BF2B831603139A00831203135708831693
:1007900003139B00831603131C158B1355309D0008
:1007A000AA309D009C148B171C11831203130800A0
:1007B000D0000008BD23840AD70AD00BD92B08002B
:1007C000D000A2238000840AD70AD00BE12B0800B6
:1007D0005908D700FC30D70DD70DD705403084001D
:0607E0000430D8230800DC
:02400E00823FEF
:00000001FF
